:02000000FC28DA
:080008000000000009000530B2
:100010009700A5309800980B0B28970B09280034FF
:10002000860083160030860083120515851005149E
:1000300005108316FF308600831205118514051400
:1000400006089C009C1705100514861F292805101A
:10005000242805104028860083160030860083126D
:1000600005118510051405108316FF3086008312D4
:1000700085140514861F3E28051039280510003404
:100080001C1C00349C1C00341C1D00349C1D0034BE
:1000900039309C079C171C082B28831310088D02ED
:1000A0000318592801308E02031859288F02031CA7
:1000B000831711088E020318612801308F02031C78
:1000C000831712088F02031C8317003410088D0752
:1000D000031C6D288E0F6D288F0A11088E070318D8
:1000E0008F0A12088F0700340730970019308400F8
:1000F0002F308000840A970B79280F30920042300D
:100100009100403090004D20990A3A3019060319A9
:10011000292A831F832866200130920086309100AF
:10012000A03090004D209A0A831F922866209201E9
:1001300027309100103090004D209B0A831F9C288F
:10014000662003309100E83090004D209C0A831F08
:10015000A52866209101643090004D209D0A831FE0
:10016000AD2866200A3090004D209E0A831FB428D7
:1001700066200D089F079F0A0034831637308100E0
:10018000103085008312851105118F0181019601C0
:10019000051505110C0897008515FA309800D6282A
:1001A00000000000000000000000000001089602AE
:1001B000031DDC280000DE2803188F0A96000000CB
:1001C00000000000980BD028970BCD28851101085E
:1001D0008E009602031CEE28031D8F0A8D018D03ED
:1001E0000515051101080E060319EF280034051442
:1001F0000720051007200034850186018316103082
:100200008500003086008312072007200720383041
:100210008600F720F720F72038302B200C302B20D9
:1002200001302B2006302B202030102020301020D1
:100230004630102052301020453010205130102010
:1002400055301020453010204E3010204330102003
:100250004530102020301020203010202030102079
:10026000203010202030102006309900C8309A002D
:1002700007209A0B3829990B362901302B2006309C
:100280002B2014308C00BD20742030301906031D43
:100290004D2930301A0603198C2982302B20023068
:1002A00097001930840030300006031D5D2920308E
:1002B0001020840A970B5329622900081020840A11
:1002C000970B5D292E301020053097000008102074
:1002D000840A970B6629203010204D3010204830BA
:1002E00010207A301020203010202030102041299A
:1002F00014308C00BD20742030301906031D4D29A8
:1003000032301A0203184D2930301A06031D8C2989
:1003100030301B060319B52982302B200530970099
:100320001930840030300006031D9C292030102035
:10033000840A970B9229A12900081020840A970BA0
:100340009C292E30102000081020840A000810205C
:10035000203010204B301020483010207A301020F0
:1003600020301020203010207829C8308C00BD208B
:10037000742030301906031D782932301A02031810
:10038000782930301A06031DC92930301B0603199D
:10039000052A82302B200430970019308400303039
:1003A0000006031DD92920301020840A970BCF297D
:1003B000DE2900081020840A970BD9292E3010203E
:1003C00000081020840A00081020840A0008102069
:1003D000203010204B301020483010207A30102070
:1003E0002030102020301020B529C8308C00BD20CE
:1003F000742030301906031DC92930301A06031D38
:10040000C92932301B020318C92982302B2007303A
:1004100097001930840030300006031D152A203063
:100420001020840A970B0B2A1A2A00081020840A2D
:10043000970B152A20301020483010207A301020D9
:1004400020301020203010202030102020301020AC
:10045000F52901302B2084302B204F3010207630AE
:1004600010206530102072301020663010206C3063
:1004700010206F3010207730102002302B204129BF
:02400E00F13F80
:1042000057344334543436345F3431345F343134CA
:104210003234303431343134323420340034503498
:1042200049344334313436344634383434342D341C
:1042300030343434203420342034003438343434AE
:104240002D34303431343434333420342034203479
:1042500020342034203420340034313432342034BB
:104260006A3461346E342034323430343134323490
:08427000203420342034003416
:00000001FF
